:020000040000FA
:04080000F1EF04F020
:1008100003B23DEF04F0F2B458EF04F09EB060EF85
:1008200004F09EB268EF04F0F2A81AEF04F0F2B2FE
:100830001CEF04F0CFEF04F0CD90F29207BC078ECE
:10084000078C9EA029EF04F00101463F29EF04F038
:10085000472B07AE34EF04F0CECF51F1CFCF52F19A
:1008600046C153F147C154F1CF6ACE6A0101466BCC
:10087000476B9E90CD80CFEF04F00392030103EE0F
:1008800000F080517F0BE92604C0EFFF802B8151DF
:10089000805D700BD8A48B8200008051815D700B4D
:1008A000D8A48B9281518019D8B40790CFEF04F06F
:1008B000F2940101383FCFEF04F0392BCFEF04F071
:1008C0009E900101463FCFEF04F0472BCFEF04F09D
:1008D0009E92C3CF48F1C4CF49F1C28207B492EFD0
:1008E00004F03AC13EF13BC13FF13CC140F13DC192
:1008F00041F151C155F152C156F153C157F154C1A3
:1009000058F1010148514E2749514F23E86A5023BD
:100910000D2E92EF04F04FC14AF150C14BF14E6BD6
:100920004F6B506B0201002FCFEF04F03C0E006FB5
:10093000D57ED5BE32D0D6CF3AF1D7CF3BF138C134
:100940003CF1E86AE8CF3DF1010147A7B3EF04F0BD
:10095000079C079E0101000E516F600E526F3D0E05
:10096000536F080E546F01013ABFC3EF04F03B67A9
:10097000C3EF04F03C67C3EF04F03D67C3EF04F03E
:10098000F288C8EF04F0F298516B526B536B546BC2
:10099000D76AD66A0101386B396BCFEF04F002C019
:1009A000E0FF005001C0D8FF1000A6B2D5EF04F060
:1009B0000CC0A9FF0BC0A8FFA69EA69CA684F29E11
:1009C000550EA76EAA0EA76EA682F28EA694A6B2A8
:1009D000E7EF04F01200A96EA69EA69CA680A85080
:1009E0001200076A0F010E0EC16E860EC06E030E56
:1009F000C26E0F01896A110E926E080E8A6EF10E98
:100A0000936E8B6A800E946EF18E818482860D6A5D
:100A10004E6B4F6B506B4A6B4B6B0F01280ED56EB4
:100A2000F28AB00ECD6E9D800101516B526B536BFB
:100A3000546B556B566B576B586B596B5A6B5B6BA2
:100A40005C6B079C079E760ECA6E9D8202013C0E6F
:100A5000006FCC6A240EAC6E0401806B816B0F01B9
:100A6000900EAB6E0F019D8A0301806B816BA26BB0
:100A70008B9207900001F28EF28C07B0DCEF0CF045
:100A80008B740301805181197F0BD8B4DCEF0CF01B
:100A900013EE00F081517F0BE126812BE7CFE8FFB9
:100AA000E00BD8B4DCEF0CF023EE82F0A2511F0B68
:100AB000D926E7CFDFFFA22BDF50780AD8A4DCEFDE
:100AC0000CF007808251720AD8B45EEF07F08251B1
:100AD000630AD8B49CEF09F08251690AD8B4D1EF07
:100AE00005F082517A0AD8B4E4EF06F08251660A22
:100AF000D8B490EF05F0D1EF09F0040114EE00F046
:100B000080517F0BE12682C4E7FF802B12000D0E7F
:100B1000826F7DEC05F00A0E826F7DEC05F012000D
:100B20008351780AD8B4AAEF05F0030183B102D04B
:100B3000829601D0828683B302D0819401D08184D1
:100B400084B102D0829A01D0828A84B302D0829882
:100B500001D082880401660E826F7DEC05F0300EB4
:100B600082B602D0E89001D0E88081B402D0E89249
:100B700001D0E882E8CF82F47DEC05F0300E82BA35
:100B800002D0E89001D0E88082B802D0E89201D08B
:100B9000E882E8CF82F47DEC05F087EC05F0D1EF38
:100BA00009F00401690E826F7DEC05F004012C0E42
:100BB000826F7DEC05F00101030E006F000E016FE6
:100BC000000E026F000E036F6BEC0FF020C182F479
:100BD0000401300E82277DEC05F021C182F404016E
:100BE000300E82277DEC05F022C182F40401300E24
:100BF00082277DEC05F023C182F40401300E8227A8
:100C00007DEC05F024C182F40401300E82277DECD6
:100C100005F025C182F40401300E82277DEC05F039
:100C200026C182F40401300E82277DEC05F027C135
:100C300082F40401300E82277DEC05F004012C0EB5
:100C4000826F7DEC05F00101040E006F000E016F54
:100C5000000E026F000E036F6BEC0FF020C182F4E8
:100C60000401300E82277DEC05F021C182F40401DD
:100C7000300E82277DEC05F022C182F40401300E93
:100C800082277DEC05F023C182F40401300E822717
:100C90007DEC05F024C182F40401300E82277DEC46
:100CA00005F025C182F40401300E82277DEC05F0A9
:100CB00026C182F40401300E82277DEC05F027C1A5
:100CC00082F40401300E82277DEC05F004012C0E25
:100CD000826F7DEC05F001010C0E006F000E016FBC
:100CE000000E026F000E036F6BEC0FF020C182F458
:100CF0000401300E82277DEC05F021C182F404014D
:100D0000300E82277DEC05F022C182F40401300E02
:100D100082277DEC05F023C182F40401300E822786
:100D20007DEC05F024C182F40401300E82277DECB5
:100D300005F025C182F40401300E82277DEC05F018
:100D400026C182F40401300E82277DEC05F027C114
:100D500082F40401300E82277DEC05F004012C0E94
:100D6000826F7DEC05F0200EF86EF76AF66A0401DA
:100D70000900F5CF82F47DEC05F00900F5CF82F48F
:100D80007DEC05F00900F5CF82F47DEC05F009005B
:100D9000F5CF82F47DEC05F00900F5CF82F47DEC0F
:100DA00005F00900F5CF82F47DEC05F00900F5CFE0
:100DB00082F47DEC05F00900F5CF82F47DEC05F0BE
:100DC00087EC05F0D1EF09F08351630AD8A4D1EF85
:100DD00009F08451610AD8A4D1EF09F085516C0A59
:100DE000D8A4D1EF09F08651410A42E08651440A65
:100DF0001BE08651420AD8B44BEF07F08651350A02
:100E0000D8B45AEF0BF08651360AD8B4AEEF0BF0D7
:100E10008651370AD8B416EF0CF08651380AD8B488
:100E200074EF0CF0D1EF09F00798079A04017A0EDD
:100E3000826F7DEC05F00401780E826F7DEC05F089
:100E40000401640E826F7DEC05F081A82FEF07F09E
:100E50000401550E826F7DEC05F034EF07F00401BC
:100E60004C0E826F7DEC05F087EC05F0D1EF09F0B8
:100E70000788079A04017A0E826F7DEC05F0040161
:100E8000410E826F7DEC05F00401610E826F7DECF6
:100E900005F025EF07F00798078A04017A0E826FA4
:100EA0007DEC05F00401420E826F7DEC05F004013B
:100EB000610E826F7DEC05F025EF07F00401720EE4
:100EC000826F7DEC05F004012C0E826F7DEC05F045
:100ED000078455C159F156C15AF157C15BF158C148
:100EE0005CF13EC142F13FC143F140C144F141C117
:100EF00045F14AC14CF14BC14DF107940101620E1D
:100F0000046F010E056F000E066F000E076F59C1CA
:100F100000F15AC101F15BC102F15CC103F1D1ECF6
:100F20000EF003BFDBEF07F00E0EEBEC04F0E8CFA2
:100F30000CF10F0EEBEC04F0E8CF0DF1100EEBEC22
:100F400004F0E8CF0EF1110EEBEC04F0E8CF0FF156
:100F50001AEC0EF059C104F15AC105F15BC106F15A
:100F60005CC107F1D1EC0EF00782DEEC0DF01AEC5B
:100F70000EF00792DEEC0DF059C100F15AC101F1FB
:100F80005BC102F15CC103F10792DEEC0DF0CC0E07
:100F9000046FE00E056F870E066F050E076FD1EC2C
:100FA0000EF000C10CF101C10DF102C10EF103C13F
:100FB0000FF114EF08F00101800E006F1A0E016F9F
:100FC000060E026F000E036F42C104F143C105F12A
:100FD00044C106F145C107F1D1EC0EF003AFF5EFC6
:100FE00007F0C8EC0FF027EF08F00E0EEBEC04F062
:100FF000E8CF0CF10F0EEBEC04F0E8CF0DF1100E82
:10100000EBEC04F0E8CF0EF1110EEBEC04F0E8CFBE
:101010000FF142C100F143C101F144C102F145C1E8
:1010200003F10782DEEC0DF00CC100F10DC101F1FE
:101030000EC102F10FC103F10101000E046F000E99
:10104000056F010E066F000E076FFFEC0EF06BECE4
:101050000FF01D6731EF08F00401200E826F34EFAE
:1010600008F004012D0E826F7DEC05F024C182F49E
:101070000401300E82277DEC05F025C182F40401C5
:10108000300E82277DEC05F004012E0E826F7DEC80
:1010900005F026C182F40401300E82277DEC05F0B4
:1010A00027C182F40401300E82277DEC05F0040193
:1010B0006D0E826F7DEC05F004012C0E826F7DECCD
:1010C00005F042C100F143C101F144C102F145C143
:1010D00003F101016BEC0FF01EC182F40401300E2C
:1010E00082277DEC05F01FC182F40401300E8227B7
:1010F0007DEC05F020C182F40401300E82277DECE6
:1011000005F021C182F40401300E82277DEC05F048
:1011100022C182F40401300E82277DEC05F023C148
:1011200082F40401300E82277DEC05F024C182F4A4
:101130000401300E82277DEC05F025C182F4040104
:10114000300E82277DEC05F026C182F40401300EBA
:1011500082277DEC05F027C182F40401300E82273E
:101160007DEC05F00401480E826F7DEC05F0040172
:101170007A0E826F7DEC05F004012C0E826F7DECFF
:1011800005F059C100F15AC101F15BC102F15CC126
:1011900003F101016BEC0FF01EC182F40401300E6B
:1011A00082277DEC05F01FC182F40401300E8227F6
:1011B0007DEC05F020C182F40401300E82277DEC25
:1011C00005F021C182F40401300E82277DEC05F088
:1011D00022C182F40401300E82277DEC05F023C188
:1011E00082F40401300E82277DEC05F024C182F4E4
:1011F0000401300E82277DEC05F025C182F4040144
:10120000300E82277DEC05F026C182F40401300EF9
:1012100082277DEC05F027C182F40401300E82277D
:101220007DEC05F00401630E826F7DEC05F0040196
:101230002C0E826F7DEC05F059C100F15AC101F10D
:101240005BC102F15CC103F101010A0E046F000EE3
:10125000056F000E066F000E076FE0EC0EF0000E3B
:10126000046F120E056F000E066F000E076FFFEC85
:101270000EF06BEC0FF01EC182F40401300E8227D9
:101280007DEC05F01FC182F40401300E82277DEC55
:1012900005F020C182F40401300E82277DEC05F0B8
:1012A00021C182F40401300E82277DEC05F022C1B9
:1012B00082F40401300E82277DEC05F023C182F414
:1012C0000401300E82277DEC05F024C182F4040174
:1012D000300E82277DEC05F004012E0E826F7DEC2E
:1012E00005F025C182F40401300E82277DEC05F063
:1012F00026C182F40401300E82277DEC05F027C15F
:1013000082F40401300E82277DEC05F00401730E97
:10131000826F7DEC05F004012C0E826F7DEC05F0F0
:10132000C8EC0FF04CC100F14DC101F1FAEC0AF02C
:1013300087EC05F0D1EF09F00401630E826F7DECBC
:1013400005F004012C0E826F7DEC05F0D6EC09F05F
:1013500004012C0E826F7DEC05F049EC0AF00401CB
:101360002C0E826F7DEC05F0C5EC0AF004012C0E0A
:10137000826F7DEC05F00101F80E006FCD0E016F5C
:10138000660E026F030E036FEBEC09F004012C0EE6
:10139000826F7DEC05F0DBEC0AF087EC05F0D1EF15
:1013A00009F00301A26B0790DCEF0CF0D8900E0E51
:1013B000EBEC04F0E8CF00F10F0EEBEC04F0E8CF1B
:1013C00001F1100EEBEC04F0E8CF02F1110EEBECA2
:1013D00004F0E8CF03F10101000E046F000E056F69
:1013E000010E066F000E076FFFEC0EF06BEC0FF0B6
:1013F0001EC182F40401300E82277DEC05F01FC16E
:1014000082F40401300E82277DEC05F020C182F4C5
:101410000401300E82277DEC05F021C182F4040125
:10142000300E82277DEC05F022C182F40401300EDB
:1014300082277DEC05F023C182F40401300E82275F
:101440007DEC05F024C182F40401300E82277DEC8E
:1014500005F025C182F40401300E82277DEC05F0F1
:1014600004012E0E826F7DEC05F026C182F404018A
:10147000300E82277DEC05F027C182F40401300E86
:1014800082277DEC05F004016D0E826F7DEC05F086
:101490001200120EEBEC04F0E8CF00F1130EEBECAF
:1014A00004F0E8CF01F1140EEBEC04F0E8CF02F108
:1014B000150EEBEC04F0E8CF03F101010A0E046F06
:1014C000000E056F000E066F000E076FE0EC0EF0C9
:1014D000000E046F120E056F000E066F000E076FF0
:1014E000FFEC0EF06BEC0FF01EC182F40401300E25
:1014F00082277DEC05F01FC182F40401300E8227A3
:101500007DEC05F020C182F40401300E82277DECD1
:1015100005F021C182F40401300E82277DEC05F034
:1015200022C182F40401300E82277DEC05F023C134
:1015300082F40401300E82277DEC05F024C182F490
:101540000401300E82277DEC05F004012E0E826F1F
:101550007DEC05F025C182F40401300E82277DEC7C
:1015600005F026C182F40401300E82277DEC05F0DF
:1015700027C182F40401300E82277DEC05F00401BE
:10158000730E826F7DEC05F012000A0EEBEC04F096
:10159000E8CF00F10B0EEBEC04F0E8CF01F10C0EFC
:1015A000EBEC04F0E8CF02F10D0EEBEC04F0E8CF29
:1015B00003F1FAEF0AF0060EEBEC04F0E8CF00F1CD
:1015C000070EEBEC04F0E8CF01F1080EEBEC04F0B1
:1015D000E8CF02F1090EEBEC04F0E8CF03F1FAEFEB
:1015E0000AF00101C8EC0FF007844AC100F14BC1B9
:1015F00001F107940101E80E046F800E056F000EE3
:10160000066F000E076FE0EC0EF0000E046F040E84
:10161000056F000E066F000E076FFFEC0EF0880ED0
:10162000046F130E056F000E066F000E076FD1ECEE
:101630000EF00A0E046F000E056F000E066F000E0E
:10164000076FFFEC0EF06BEC0FF001011D672EEF42
:101650000BF00401200E826F31EF0BF004012D0E10
:10166000826F7DEC05F024C182F40401300E8227E4
:101670007DEC05F025C182F40401300E82277DEC5B
:1016800005F026C182F40401300E82277DEC05F0BE
:1016900004012E0E826F7DEC05F027C182F4040157
:1016A000300E82277DEC05F00401430E826F7DEC45
:1016B00005F0120087C31EF188C31FF189C320F112
:1016C0008AC321F18BC322F18CC323F18DC324F192
:1016D0008EC325F190C326F191C327F1010115ECCA
:1016E00010F08DEC0FF00101000E046F000E056F7D
:1016F000010E066F000E076FE0EC0EF00E0E0C6E82
:1017000000C10BF0D5EC04F00F0E0C6E01C10BF014
:10171000D5EC04F0100E0C6E02C10BF0D5EC04F009
:10172000110E0C6E03C10BF0D5EC04F004017A0E1F
:10173000826F7DEC05F004012C0E826F7DEC05F0CC
:101740000401350E826F7DEC05F004012C0E826FD2
:101750007DEC05F0D6EC09F034EF07F087C31EF1FD
:1017600088C31FF189C320F18AC321F18BC322F101
:101770008CC323F18DC324F18EC325F190C326F1D0
:1017800091C327F1010115EC10F08DEC0FF0880EDC
:10179000046F130E056F000E066F000E076FD5EC79
:1017A0000EF0000E046F040E056F000E066F000EA3
:1017B000076FE0EC0EF00101E80E046F800E056F7C
:1017C000000E066F000E076FFFEC0EF00A0E0C6E97
:1017D00000C10BF0D5EC04F00B0E0C6E01C10BF048
:1017E000D5EC04F00C0E0C6E02C10BF0D5EC04F03D
:1017F0000D0E0C6E03C10BF0D5EC04F004017A0E53
:10180000826F7DEC05F004012C0E826F7DEC05F0FB
:101810000401360E826F7DEC05F004012C0E826F00
:101820007DEC05F0C5EC0AF034EF07F087C31EF13C
:1018300088C31FF189C320F18AC321F18BC322F130
:101840008CC323F18DC324F18FC325F190C326F1FE
:1018500091C327F1010115EC10F08DEC0FF0000E93
:10186000046F120E056F000E066F000E076FE0EC9E
:101870000EF001010A0E046F000E056F000E066FD8
:10188000000E076FFFEC0EF0120E0C6E00C10BF095
:10189000D5EC04F0130E0C6E01C10BF0D5EC04F086
:1018A000140E0C6E02C10BF0D5EC04F0150E0C6E8C
:1018B00003C10BF0D5EC04F004017A0E826F7DECCD
:1018C00005F004012C0E826F7DEC05F00401370E4B
:1018D000826F7DEC05F004012C0E826F7DEC05F02B
:1018E00049EC0AF034EF07F087C31EF188C31FF1FB
:1018F00089C320F18AC321F18BC322F18CC323F168
:101900008DC324F18EC325F190C326F191C327F135
:10191000010115EC10F08DEC0FF0880E046F130E22
:10192000056F000E066F000E076FD5EC0EF0000E6F
:10193000046F040E056F000E066F000E076FE0ECDB
:101940000EF00101E80E046F800E056F000E066FA9
:10195000000E076FFFEC0EF0060E0C6E00C10BF0D0
:10196000D5EC04F0070E0C6E01C10BF0D5EC04F0C1
:10197000080E0C6E02C10BF0D5EC04F0090E0C6ED3
:1019800003C10BF0D5EC04F004017A0E826F7DECFC
:1019900005F004012C0E826F7DEC05F00401380E79
:1019A000826F7DEC05F004012C0E826F7DEC05F05A
:1019B000DBEC0AF034EF07F081A89AEF0DF007A8EE
:1019C00053EF0DF00101800E006F1A0E016F060E2D
:1019D000026F000E036F3EC104F13FC105F140C12B
:1019E00006F141C107F1D1EC0EF003BF9AEF0DF003
:1019F000D8EC0DF03EC100F13FC101F140C102F150
:101A000041C103F10782DEEC0DF00CC104F10DC100
:101A100005F10EC106F10FC107F1F80E006FCD0EF2
:101A2000016F660E026F030E036FD1EC0EF00E0E07
:101A30000C6E00C10BF0D5EC04F00F0E0C6E01C162
:101A40000BF0D5EC04F0100E0C6E02C10BF0D5ECCF
:101A500004F0110E0C6E03C10BF0D5EC04F00784FA
:101A60000101C8EC0FF04AC100F14BC101F107942C
:101A70000A0E0C6E00C10BF0D5EC04F00B0E0C6ED0
:101A800001C10BF0D5EC04F00C0E0C6E02C10BF092
:101A9000D5EC04F00D0E0C6E03C10BF0D5EC04F088
:101AA00007989AEF0DF007AA9AEF0DF0078401014D
:101AB000C8EC0FF04AC100F14BC101F10794060ECA
:101AC0000C6E00C10BF0D5EC04F0070E0C6E01C1DA
:101AD0000BF0D5EC04F0080E0C6E02C10BF0D5EC47
:101AE00004F0090E0C6E03C10BF0D5EC04F0078472
:101AF00055C100F156C101F157C102F158C103F1BE
:101B00000794120E0C6E00C10BF0D5EC04F0130E0E
:101B10000C6E01C10BF0D5EC04F0140E0C6E02C17A
:101B20000BF0D5EC04F0150E0C6E03C10BF0D5ECE8
:101B300004F0079A0401805181197F0B0BE09EA8E5
:101B400009D014EE00F081517F0BE126E750812B84
:101B50000F01AD6E3DEF05F00CC100F10DC101F1BB
:101B60000EC102F10FC103F1000E046F000E056FEC
:101B7000010E066F000E076FFFEC0EF01DA1D7EFF0
:101B80000DF01451D8B4D7EF0DF00CC100F10DC118
:101B900001F10EC102F10FC103F1000E046F000E3E
:101BA000056F0A0E066F000E076FFFEC0EF01200B5
:101BB00001010C6B0D6B0E6B0F6B120001010053DA
:101BC00005E1015303E1025301E1002BA1EC0EF00A
:101BD000C8EC0FF02C51006F2D51016F420E046FB5
:101BE0004B0E056F000E066F000E076FE0EC0EF057
:101BF00000C104F101C105F102C106F103C107F101
:101C00000CC100F10DC101F10EC102F10FC103F1D0
:101C100007B20FEF0EF0D5EC0EF011EF0EF0D1EC95
:101C20000EF000C10CF101C10DF102C10EF103C1B2
:101C30000FF11200C8EC0FF04CC100F14DC101F1E1
:101C4000060EEBEC04F0E8CF04F1070EEBEC04F029
:101C5000E8CF05F1080EEBEC04F0E8CF06F1090E31
:101C6000EBEC04F0E8CF07F1D1EC0EF000C118F175
:101C700001C119F102C11AF103C11BF1290E046F50
:101C8000000E056F000E066F000E076FE0EC0EF001
:101C9000EE0E046F430E056F000E066F000E076F09
:101CA000D5EC0EF018C104F119C105F11AC106F105
:101CB0001BC107F1E0EC0EF000C110F101C111F100
:101CC00002C112F103C113F1120EEBEC04F0E8CFE4
:101CD00004F1130EEBEC04F0E8CF05F1140EEBEC7D
:101CE00004F0E8CF06F1150EEBEC04F0E8CF07F1B5
:101CF0000D0E006F000E016F000E026F000E036FDD
:101D0000E0EC0EF0180E046F000E056F000E066F6B
:101D1000000E076FFFEC0EF010C104F111C105F1C8
:101D200012C106F113C107F1D5EC0EF06A0E046F73
:101D30002A0E056F000E066F000E076FD1EC0EF035
:101D40001200BF0EFA6E200E2D6F2C6BD89000374C
:101D5000013702370337D8B0B2EF0EF02D2FA7EFBF
:101D60000EF02C072D070353D8B412000331070BD4
:101D70008009326F03390F0B010F2C6F80EC5FF07D
:101D8000336F2C0580EC5FF0335D335F2C6B3233A7
:101D9000D8B02C272C3332A9C7EF0EF033512C27A3
:101DA0001200EDEC0FF0D8B0120003510719286FA4
:101DB000B0EC0FF0D8900751031928AF800F120034
:101DC000286BD4EC0FF0D8A0EAEC0FF0D8B01200DA
:101DD000BFEC0FF0C8EC0FF01F0E296F00EC10F0F5
:101DE0000B35D8B0B0EC0FF0D8A00335D8B0120046
:101DF000292FEEEF0EF028B1D7EC0FF01200286B70
:101E000004510511061107110008D8A0D4EC0FF0F9
:101E1000D8A0EAEC0FF0D8B01200086B096B0A6B7F
:101E20000B6B00EC10F01F0E296F00EC10F0075147
:101E30000B5DD8A428EF0FF006510A5DD8A428EF57
:101E40000FF00551095DD8A428EF0FF00451085D8B
:101E5000D8A03BEF0FF00451085F0551D8A0053D15
:101E6000095F0651D8A0063D0A5F0751D8A0073D7B
:101E70000B5FD8900081292F15EF0FF028B1D7EC18
:101E80000FF0286BD4EC0FF0D89004EC10F0075151
:101E90000B5DD8A458EF0FF006510A5DD8A458EF97
:101EA0000FF00551095DD8A458EF0FF00451085DFB
:101EB000D8A067EF0FF0003F67EF0FF0013F67EF2B
:101EC0000FF0023F67EF0FF0032BD8B4120028B1D8
:101ED000D7EC0FF012000101286BD4EC0FF0D8B052
:101EE000120009EC10F0200E296F0037013702377D
:101EF000033711EE27F00A0E2A6FE7360A0EE75C69
:101F0000D8B0E76EE5522A2F7DEF0FF0292F75EF3D
:101F10000FF028B11D81D890120001010A0E286F20
:101F2000200E296F11EE1DF028512A6F0A0ED8904D
:101F3000E652D8B0E726E7322A2F98EF0FF00333A6
:101F4000023301330033292F92EF0FF0E750FF0FD8
:101F5000D8A00335D8B012001DB1D7EC0FF0120095
:101F6000045100270551D8B0053D01270651D8B0CE
:101F7000063D02270751D8B0073D03271200005144
:101F8000086F0151096F02510A6F03510B6F120064
:101F90000101006B016B026B036B12000101046B0A
:101FA000056B066B076B12000335D8A012000351B6
:101FB000800B001F011F021F031F003FE7EF0FF000
:101FC000013FE7EF0FF0023FE7EF0FF0032B282B65
:101FD000032512000735D8A012000751800B041FFB
:101FE000051F061F071F043FFDEF0FF0053FFDEF24
:101FF0000FF0063FFDEF0FF0072B282B07251200EF
:102000000037013702370337083709370A370B37EC
:1020100012001D6B1E6B1F6B206B216B226B236BE1
:10202000246B256B266B276B12001E510F0B1E6F46
:102030001F510F0B1F6F20510F0B206F21510F0BE2
:10204000216F22510F0B226F23510F0B236F24514D
:102050000F0B246F25510F0B256F26510F0B266F89
:0820600027510F0B276F12003E
:10BF0000E844F926000C160C2B0C3F0C520C640C68
:10BF1000760C860C960CA50CB30CC10CCF0CDC0C6B
:06BF2000E80CF40C000C1B
:00000001FF
